:100000000C9434020C948E020C94BB020C945C028F
:100010000C945C020C945C020C945C020C945C02E8
:100020000C945C020C945C020C945C020C945C02D8
:100030000C945C020C945C020C945C020C945C02C8
:100040000C945C020C945C020C94E8020C945C022C
:100050000C94A6190C945C020C945C020C945C0247
:100060000C945C020C945C020C945C020C945C0298
:100070000C945C020C945C020C945C02DF17671811
:100080006B18A818CC17BE187118451757174A17C0
:100090005B1785179017BE18DB17BE18BE18BD1763
:1000A0004F17B417BE1852178A18BE180918A1178F
:1000B0009718F1176017A617AB17B41800002100A6
:1000C000240027002A0000002200250028002B0021
:1000D000000020002300260029000303030403027C
:1000E00002040404040403030101010101010101EC
:1000F000030202020202020102044008100804087E
:1001000020108010400102040810204080200102CD
:1001100004204080000000070002010000030406E4
:1001200000000000000000000000000000000000CF
:1001300000687474703A2F2F6269746C6173682E52
:100140006E65740D0A536565204C4943454E534511
:1001500020666F72206C6963656E73652C20524552
:1001600041444D4520666F7220686F77746F0D0AA9
:1001700050696E733A2064302D32322C61302D324A
:100180003220205661726961626C65733A20612D7C
:100190007A2C20333220626974206C6F6E6720697C
:1001A0006E7465676572730D0A4F70657261746F66
:1001B00072733A202B202D202A202F20282029203E
:1001C0003C203C3D203E203E3D203D3D20213D2029
:1001D0003C3C203E3E2021205E2026207C202B2BF4
:1001E000202D2D203A3D0D0A436F6D6D616E6473B5
:1001F0003A2000007072696E7420226269746C612A
:1002000073682068657265212076302E3935612D3E
:1002100052432028632920323030392042696C6CE7
:1002200020526F79202D747970652048454C502DEF
:10023000222C667265652C22627974657320667261
:1002400065652200010102020301030101010201AF
:100250000202000105020002020203020100040181
:100260000100000101616273006172006177006248
:10027000617564006265657000627574746F6E7399
:1002800000636F6E73747261696E0064656C61798E
:100290000064720064750064770065720065770021
:1002A000666C6173680066726565006B6579006DE8
:1002B0006170006D6178006D696C6C6973006D69C7
:1002C0006E006D6F76650070696E6D6F64650070AD
:1002D000756C7365696E0072616E64320072616E76
:1002E000646F6D0073610073686966746F75740084
:1002F0007369676E00736E6F6F7A65007372007357
:10030000796D730075737200776865656C000065C0
:10031000787065637465642000756E6578706563D8
:1003200074656420006D697373696E67200073746F
:1003300072696E670020756E646572666C6F770017
:10034000206F766572666C6F77005E43005E4200D8
:100350005E5500657870006F70003A7862792B2DD9
:100360002A2F00656F6600766172006E756D62659A
:1003700072002900736176656400656570726F6D47
:10038000003A3D22003E20006C696E6500636861A2
:100390007200737461636B007374617274757000C2
:1003A00069640070726F6D7074000D0A46756E633B
:1003B00074696F6E733A006F6F7073000034444459
:1003C000444004404444444444444444440877473B
:1003D000857778787711111111118788844222224C
:1003E0002222222222222222222224447242222259
:1003F00022222222222222222222248474626F6F4D
:10040000740068656C70006966006C7300706565E7
:1004100070007072696E7400707300726D00727596
:100420006E0073746F700073776974636800776827
:10043000696C6500001A1C101D1B1E181617191F69
:100440001126267C7C3D3D213D2B2B2D2D3A3D3E1A
:100450003D3E3E3C3D3C3C00060708090C0D1405A2
:100460000B040A00021BC11D11241FBECFEFD8E0F0
:10047000DEBFCDBF12E0A0E0B1E0E0E0F9E502C0F0
:1004800005900D92AC33B107D9F714E0ACE3B2E0BC
:1004900001C01D92A33AB107E1F714E0C8E6D4E029
:1004A00004C02297FE010E945E2CC436D107C9F712
:1004B0000E94A1140C947E2C0C9400008230E8F46D
:1004C000E82FF0E0EE0FFF1FE45CFD4F71836083C7
:1004D000813041F0809169008C7F842B809369008A
:1004E000E89A089580916900440F551F440F551FE5
:1004F000837F842B80936900E99A0895823068F4A1
:10050000813011F0E89801C0E998E82FF0E0EE0F93
:10051000FF1FE45CFD4F1182108208951F920F921D
:100520000FB60F9211242F933F934F935F936F93C6
:100530007F938F939F93AF93BF93EF93FF9380919C
:100540003C0290913D02009729F0E0913C02F0912D
:100550003D020995FF91EF91BF91AF919F918F91CE
:100560007F916F915F914F913F912F910F900FBEAF
:100570000F901F9018951F920F920FB60F92112493
:100580002F933F934F935F936F937F938F939F939B
:10059000AF93BF93EF93FF9380913E0290913F0200
:1005A000009729F0E0913E02F0913F020995FF91FA
:1005B000EF91BF91AF919F918F917F916F915F91DB
:1005C0004F913F912F910F900FBE0F901F90189554
:1005D0001F920F920FB60F9211242F938F939F9318
:1005E000AF93BF938091400290914102A09142024B
:1005F000B09143020196A11DB11D809340029093DA
:100600004102A0934202B093430280914402909130
:100610004502A0914602B09147028050904CAF4FE6
:10062000BF4F8093440290934502A0934602B0933B
:10063000470227C08091440290914502A091460252
:10064000B091470280529E44A040B0408093440243
:1006500090934502A0934602B093470280914802CE
:1006600090914902A0914A02B0914B020196A11DBE
:10067000B11D8093480290934902A0934A02B0931F
:100680004B028091440290914502A0914602B091A4
:10069000470281322EE4920720E0A20720E0B20751
:1006A00048F6BF91AF919F918F912F910F900FBE00
:1006B0000F901F9018958FB7F894209148023091B1
:1006C000490240914A0250914B028FBFB901CA01C1
:1006D00008956FB7F89426B530E040E050E0A89B4D
:1006E00009C0211531054105510521F420E031E013
:1006F00040E050E08091400290914102A09142027E
:10070000B09143026FBFBA2FA92F982F8827820F6D
:10071000931FA41FB51F9C01AD01220F331F441F5F
:10072000551F280F391F4A1F5B1FB901CA010895C1
:10073000EF92FF920F931F937B018C018FB7F89478
:10074000209148023091490240914A0250914B0257
:100750008FBF6FB7F8948091480290914902A091A1
:100760004A02B0914B026FBF821B930BA40BB50BD7
:10077000E816F9060A071B0760F71F910F91FF9013
:10078000EF900895019751F0880F991F880F991FD6
:1007900002972FB7F8940197F1F72FBF0895789437
:1007A00084B5826084BD84B5816084BD85B5826076
:1007B00085BD85B5816085BDEEE6F0E08081816014
:1007C0008083E1E8F0E080818260808380818160C5
:1007D0008083E0E8F0E0808181608083E1EBF0E0FD
:1007E000808184608083E0EBF0E0808181608083A1
:1007F000EAE7F0E08081846080838081826080838A
:100800008081816080838081806880831092C100B4
:10081000089580930001089587709091000192954A
:10082000990F990F907C982B90937C0080917A007F
:10083000806480937A0080917A0086FDFCCF2091BD
:10084000780030917900932F80E030E0282B392B0D
:10085000C90108951F93CF93DF93182FEB0161E037
:100860000E948304E12FF0E0EC5EFE4F8491833020
:1008700051F480918000806880938000D09389003B
:10088000C09388003CC0843051F480918000806225
:1008900080938000D0938B00C0938A0030C0813059
:1008A00039F4209729F184B5806884BDC7BD27C07D
:1008B000823039F42097E1F084B5806284BDC8BDF0
:1008C0001EC0863041F48091B00080688093B000F3
:1008D000C093B30014C0873041F48091B0008062AF
:1008E0008093B000C093B4000AC0C038D1051CF496
:1008F000812F60E002C0812F61E00E94A204DF919D
:10090000CF911F910895282F30E0C90189509F4F42
:10091000FC019491F901E652FF4FE491EE2389F036
:10092000F0E0EE0FFF1FE454FF4FA591B491662352
:1009300029F48C91909589238C9308958C91892B1F
:100940008C930895482F50E0CA018C5E9E4FFC01A5
:1009500094919A0129503F4FF9012491FA01E652EE
:10096000FF4FE491EE23C9F1992331F1933021F443
:10097000909180009F7705C0943031F49091800071
:100980009F7D9093800018C0913019F494B59F77A3
:1009900004C0923021F494B59F7D94BD0DC0963073
:1009A00021F49091B0009F7705C0973029F4909181
:1009B000B0009F7D9093B000F0E0EE0FFF1FEA5370
:1009C000FF4FA591B491662329F48C912095822341
:1009D0008C9308958C91822B8C930895282F30E06E
:1009E000C9018C5E9E4FFC019491A90149505F4F53
:1009F000FA014491F901E652FF4FE491EE2319F414
:100A000020E030E036C0992331F1933021F4909109
:100A100080009F7705C0943031F4909180009F7DD5
:100A20009093800018C0913019F494B59F7704C05A
:100A3000923021F494B59F7D94BD0DC0963021F481
:100A40009091B0009F7705C0973029F49091B00045
:100A50009F7D9093B000F0E0EE0FFF1FE053FF4F3B
:100A6000A591B4918C9120E030E0842311F021E035
:100A700030E0C9010895AF92BF92CF92DF92FF920A
:100A80000F931F93962F682F70E0FB01E950FF4FE3
:100A9000149166527F4FFB01F490992311F0012FBE
:100AA00001C000E0CA01B90124E130E040E050E0BB
:100AB0000E94A22B5B016C0134E0D694C794B794DA
:100AC000A7943A95D1F78F2D90E0880F991F805306
:100AD0009F4F20E030E040E050E0FC01A591B49150
:100AE0000AC02A153B054C055D0509F43DC02F5F82
:100AF0003F4F4F4F5F4F6C916123601791F30AC0D6
:100B00002A153B054C055D0579F12F5F3F4F4F4F8F
:100B10005F4F03C0FC01A591B4916C9161236017F4
:100B200079F720E030E040E050E0FC01A591B4917D
:100B300004C02F5F3F4F4F4F5F4F8C918123801731
:100B4000C1F3CA01B9012AE030E040E050E00E9460
:100B5000A22B605F7F4F8F4F9F4F24E130E040E03A
:100B600050E00E94D42B04C020E030E040E050E090
:100B7000B901CA011F910F91FF90DF90CF90BF90F4
:100B8000AF900895AF92BF92CF92DF92FF920F93F2
:100B90001F93CF93DF93082F162FF42EC0E0D0E0E1
:100BA000C22EDD2487E0A82EB12CFF2041F4B6012F
:100BB0000C2E02C0759567950A94E2F70AC0B5013C
:100BC0006C1B7D0BC60102C0959587956A95E2F76F
:100BD000BC016170802F0E94A204812F61E00E94FD
:100BE000A204812F60E00E94A2042196C830D105A2
:100BF000E1F6DF91CF911F910F91FF90DF90CF90A1
:100C0000BF90AF900895E0914D02F0914E0292E0B6
:100C1000EE39F90710F080E008958193F0934E02C9
:100C2000E0934D0281E00895892F8095881F8827E1
:100C3000881F08959C013068C90108959C013F7781
:100C4000C9010895FB010CC0F999FECF92BD81BD89
:100C5000F89A20B5322F31503E3F28F40196219367
:100C60004150504089F7108208959C010AC0F999BB
:100C7000FECF32BD21BDF89A80B58F3F41F42F5F82
:100C80003F4F83E02F3F380794F32FEF3FEFC90129
:100C900008959C010AC0F999FECF32BD21BDF89A92
:100CA00080B58F3F41F02F5F3F4F83E02F3F3807E4
:100CB00094F32FEF3FEFC90108959C010DC0F999FE
:100CC000FECF32BD21BDF89A80B58F3F69F08823F1
:100CD00019F42F5F3F4F08C02F5F3F4F83E02F3F36
:100CE00038076CF32FEF33E0C901089512C0F9996A
:100CF000FECF92BD81BDF89A40B550E0332727FD65
:100D000030954217530711F080E0089501966F5F08
:100D10007F4FFB012081222351F7F999FECF92BD2D
:100D200081BDF89A90B580E0992309F481E0089597
:100D3000EF92FF920F931F93CF93DF938C0180E08C
:100D400090E00E943506EC012FEF8F3F920781F073
:100D5000B8010E947606882359F4CE010E945D06F0
:100D60000E945D0633E08B3F93075CF3CFEFDFEF2C
:100D7000CE01DF91CF911F910F91FF90EF900895D9
:100D80000E9498069C0197FD03C00E945D069C018D
:100D9000C90108950EC0F999FECF6F5F7F4F1FBA4A
:100DA00092BD81BD20BD0FB6F894FA9AF99A0FBE94
:100DB0000196482F392FFB012081222361F7F999F1
:100DC000FECF1FBA842F932F92BD81BD10BC0FB6EA
:100DD000F894FA9AF99A0FBE08959C019FEFF99939
:100DE000FECF32BD21BDF89A80B58F3F91F02F5FC5
:100DF0003F4FF999FECF1FBAA9014150504052BD53
:100E000041BD90BD0FB6F894FA9AF99A0FBE8823A7
:100E100031F7C90108950E94980697FD04C00E9409
:100E2000ED060E94ED0608958091AC029091AD020E
:100E3000A091AE02B091AF020196A11DB11D8093A9
:100E4000AC029093AD02A093AE02B093AF020895AE
:100E5000EF92FF920F931F932091AC023091AD025D
:100E60004091AE025091AF0279018A010894E11CD1
:100E7000F11C011D111DE092AC02F092AD02009335
:100E8000AE021093AF02F999FECF1FBA32BD21BD59
:100E900080BD0FB6F894FA9AF99A0FBE1F910F9180
:100EA000FF90EF900895DF93CF9300D0CDB7DEB7DA
:100EB0009E01225A3440C9010F900F90CF91DF91CB
:100EC00008958F7121E030E002C0220F331F8A9510
:100ED000E2F7442737FD4095542F809115019091FA
:100EE0001601A0911701B091180182279327A4271A
:100EF000B5278093150190931601A0931701B09325
:100F000018010895E0E0F0E009950895982F87FF13
:100F100002C084E00895E82FE695F0E0E354FC4F2A
:100F2000849190FF02C08F70089582958F7008950C
:100F30008EB38C3391F08EB3843079F08EB38830D9
:100F400061F08EB3893049F08EB38E3331F09EB3A9
:100F500080E0953019F481E0089581E00895982F9C
:100F600090539A3038F09153963020F090E08154AD
:100F7000863008F491E0892F08958091BD02909108
:100F8000BE02A091BF02B091C0020196A11DB11D89
:100F90008093BD029093BE02A093BF02B093C002A3
:100FA0008AB50E948607E82FF0E0EE0FFF1FEF5F83
:100FB000FE4F0190F081E02D09950895E091A50282
:100FC000F091A602F7FD03C080818ABD0895F999CA
:100FD000FECFFF77F2BDE1BDF89A80B58ABD8AB534
:100FE0008F3F09F41ABC08958AB5809313011092BB
:100FF00014010895809113019091140197FD08C088
:101000008ABD8FEF9FEF909314018093130134C03A
:10101000E091A502F091A602F7FD0FC08081882320
:1010200029F03196F093A602E093A502E091A50283
:10103000F091A60280818ABD1FC0FF77F999FECF8B
:10104000F2BDE1BDF89A80B58ABD8AB58823A1F0CA
:101050008AB58F3F89F03196F999FECFF2BDE1BD97
:10106000F89A80B58ABDF068F093A602E093A502D5
:101070008AB58F3F09F41ABC8AB508959093A602E9
:101080008093A5020E94DE07089590680E943E08A2
:1010900008951092C1020895FC01918190538281BC
:1010A000882311F4892F08958053990F292F220F37
:1010B000220F290F820F0895E82FF0E0EE0FFF1F97
:1010C000EE0FFF1FEE51FD4F408351836283738308
:1010D0000895E82FF0E0EE0FFF1FEE0FFF1FEE5117
:1010E000FD4F60817181828193810895E82FF0E046
:1010F000EE0FFF1FEE0FFF1FEE51FD4F20813181DC
:10110000428153812F5F3F4F4F4F5F4F2083318389
:1011100042835383B901CA01089502C00E94FA07AD
:101120008AB50E9486078823C9F30E94BD070895E7
:101130008AB58EBB0E94FA0780E0A1E4B4E0FD010D
:101140009491992321F19D012F5F3F4FF901249143
:101150006EB370E0492F552747FD5095641775070A
:1011600099F44AB550E0332727FD309542175307CD
:1011700059F4E82FFF27E7FDF095E85AFB4FE4917B
:10118000EEBB0E94FA07089512968F5FD8CF08959C
:101190008AB58EBB0E94FA0708958FE08EBB089532
:1011A00010924A0308958430910538F4FC01EE0F43
:1011B000FF1FE257FC4F118210820895F999FECF6C
:1011C0001FBA92BD81BD60BD0FB6F894FA9AF99A24
:1011D0000FBE0895F999FECF92BD81BDF89A80B5F2
:1011E000089520918B03222371F0E0918D03F0E0AC
:1011F000EE0FFF1FEE0FFF1FEA56FC4F6083718357
:101200008283938308950E949803089588E0EEE80E
:10121000F3E0DF011D928A95E9F708950E9406091F
:1012200080E090E02FEFF999FECF1FBA92BD81BD0B
:1012300020BD0FB6F894FA9AF99A0FBE019634E0E1
:101240008030930781F70895CF92DF92EF92FF925B
:101250000F931F93CF93DF93082F80914A03E82FBA
:10126000F0E0EE0FFF1FE55BFC4FC081D18160E035
:101270000E94A2047E01CE010E94C20318E00AC0AF
:10128000602F617080914A030E94A204C7010E94EE
:10129000C20306951150A0F780914A0361E00E94B5
:1012A000A204CE01880F991F0E94C203DF91CF9143
:1012B0001F910F91FF90EF90DF90CF900895682FCE
:1012C00080914A03882329F481E594E00E94411B20
:1012D0000895862F0E94240908958F929F92AF92BD
:1012E000BF92CF92DF92EF92FF920F931F93DF9303
:1012F000CF93CDB7DEB7A0970FB6F894DEBF0FBE81
:10130000CDBF7B018C01611571058105910521F42B
:1013100080E30E945F0935C06E010894C11CD11C96
:10132000842E9924AA24BB24C801B701A5019401E5
:101330000E94D42BF60161936F01C801B701A5018A
:1013400094010E94D42BE22EF32E042F152FE114CA
:10135000F1040105110541F70AC0F60180818A30C8
:1013600014F4805D01C0895C0E945F0904C07E01A5
:101370000894E11CF11C0894C108D108CE14DF04C4
:1013800060F7A0960FB6F894DEBF0FBECDBFCF9129
:10139000DF911F910F91FF90EF90DF90CF90BF9062
:1013A000AF909F908F90089542E00E946D0908953C
:1013B00040E10E946D090895EF92FF920F931F93F1
:1013C0007B018C0197FF0BC08DE20E945F09109595
:1013D0000095F094E094E11CF11C011D111DC80161
:1013E000B7014AE00E946D091F910F91FF90EF90A5
:1013F00008958AE00E945F098DE00E945F090895C8
:10140000CF93DF93EC0103C021960E945F0988818E
:101410008823D1F7DF91CF910895EF92FF920F9338
:101420001F93CF93DF93E12CE0EEFE2E012D112DC3
:10143000C0E0D0E0CE018F739070009749F40E9415
:10144000F909C801B7010E94D8098AE30E945F091F
:10145000CE0187709070009719F480E20E945F09B6
:10146000CE0183709070009719F480E20E945F09AA
:10147000F999FECFD2BDC1BDF89A80B5882311F489
:101480008CE507C08F3F11F48EE203C0803208F470
:101490008EE50E945F0921960894E11CF11C011D54
:1014A000111D84E0C030D80709F0C4CF0E94F909AB
:1014B000DF91CF911F910F91FF90EF900895EF92E0
:1014C000FF921F93CF93DF93E82EE7017E01F92E61
:1014D000E70101C02196F999FECFD2BDC1BDF89AAE
:1014E00010B5812F81508E3FE8F5123229F48CE53A
:1014F0000E945F0982E21BC01C3529F48CE50E9422
:101500005F098CE514C01A3029F48CE50E945F094C
:101510008EE60DC0193029F48CE50E945F0984E73E
:1015200006C01D3039F48CE50E945F0982E70E94F5
:101530005F09D0CF812F8052803690F08CE50E94D9
:101540005F0988E70E945F09103118F480E30E9468
:101550005F09612F70E080E090E00E94D809BACF67
:10156000812FE5CFDF91CF911F91FF90EF900895EC
:10157000EF92FF920F931F93CF93DF93A4E0EA2E95
:10158000F12CC0E0D0E08E01000F111F02571C4F5C
:10159000F801808191810097A9F0BE01882777FD2D
:1015A0008095982F0E94DC098AE30E945F0980E2FF
:1015B0000E945F09F801808191819F770E945F0AF4
:1015C0000E94F90921960894E108F108E114F10458
:1015D000D1F6DF91CF911F910F91FF90EF90089579
:1015E000CF93DF93C091A502D091A602D7FD0EC084
:1015F000CF54D24004C080E20E945F092197D7FFF8
:10160000FACF8EE50E945F090E94F909DF91CF9120
:1016100008951F93CF93DF93EC01FE0114911F3FB8
:1016200089F02196112341F4FE018491882351F021
:1016300080E20E945F0902C0103679F3812F0E9478
:101640005F09EBCFDF91CF911F9108959F92AF92E9
:10165000BF92CF92DF92EF92FF920F931F93CF939F
:10166000DF93962E59016A01C801B7010E94A22B8F
:1016700028EE33E040E050E00E94D42BE22EF32E1F
:10168000042F152F60E271EA87E090E0A601950132
:101690000E94D42B59016A0189EF9FEFAFEFBFEF92
:1016A000A80EB91ECA1EDB1E892D61E00E948304AC
:1016B000E501219713C0892D61E00E94A204C501B4
:1016C0000E94C203892D60E00E94A204CE010E9404
:1016D000C2030894E108F10801091109E114F104B9
:1016E0000105110541F7DF91CF911F910F91FF90F7
:1016F000EF90DF90CF90BF90AF909F900895EF92C2
:10170000FF920F931F93CF93DF938AB590E0C0971A
:10171000AA2797FDA095BA2F8093A7029093A802BD
:10172000A093A902B093AA02CAE0D0E00E94FA07EF
:10173000992787FD90950E94762C8ABD8AB58837B7
:1017400019F4C0E1D0E0F2CF8AB590E0C0978A30BA
:10175000910548F4EAB4FF2400E010E080ED9FEF2B
:10176000AFEFBFEF11C0CA30D10571F18AB5813634
:1017700058F18AB5873640F5EAB4FF2400E010E05E
:1017800089EA9FEFAFEFBFEFE80EF91E0A1F1B1F9C
:10179000BE01882777FD8095982F2091A702309170
:1017A000A8024091A9025091AA020E94A22BE60E23
:1017B000F71E081F191FE092A702F092A8020093DB
:1017C000A9021093AA02B2CF81E08EBBDF91CF9124
:1017D0001F910F91FF90EF900895982F90539A309A
:1017E00010F4892F0895992787FD90950E94762CF3
:1017F00087550895EF92FF921F93CF93DF93182F91
:10180000C0E0D0E012C07E01B4E0EE0CFF1CBA953F
:10181000E1F78AB50E94ED0BC82FDD27C7FDD095F3
:10182000CE0DDF1D0E94FA071150112361F7CE0182
:10183000DF91CF911F91FF90EF900895FF920F934A
:101840001F93CF93DF938C01EB01F42E1092A7022C
:101850001092A8021092A9021092AA0225C0C801F3
:10186000BE010E944D2B009711F481E022C0FF20A1
:1018700011F097FD1DC08091A7029091A802A09140
:10188000A902B091AA020196A11DB11D8093A702E1
:101890009093A802A093A902B093AA02CE010E943D
:1018A000562B0196C80FD91FFE0184918823B9F6E3
:1018B00080E0DF91CF911F910F91FF900895EF92FB
:1018C000FF921F93CF93DF93182FCFE0D3E007C091
:1018D000CE010E94562B0196C80FD91F115011231B
:1018E000B9F7CE01DF91CF911F91FF90EF9008954E
:1018F000CF93DF930E945F0CEC01FE01219684914F
:10190000882319F00E945F09F8CFDF91CF910895E5
:101910000E94780C0E94F9090895DF93CF9300D0BC
:10192000CDB7DEB78093A3026093A40210924A035E
:101930006A8389830E94F00A89810E94780C6A81F7
:10194000662319F0862F0E94880C86EB93E061E0F5
:1019500070E00E942C2B65E00E948D0C0895EF92A0
:10196000FF920F931F93CF93DF937A018B01209106
:101970008E0330918F032115310519F4C0E0D0E0BA
:1019800021C020919003309191032115310519F464
:10199000C1E0D0E017C0209192033091930321154C
:1019A000310519F4C2E0D0E00DC0209194033091CC
:1019B00095032115310521F088E10E94AB0C1CC074
:1019C000C3E0D0E0FE01EE0FFF1FE257FC4F918312
:1019D00080830E945B03CC0FDD1FCC0FDD1FFE0157
:1019E000EA55FC4F6083718382839383CA56DC4F30
:1019F000E882F9820A831B83DF91CF911F910F91B7
:101A0000FF90EF900895DF93CF9300D0CDB7DEB76E
:101A100081E594E00E94A41A882381F081E594E096
:101A20000E94BA1A8330910549F486E00E94880C1E
:101A300086EB93E061E070E00E942C2BCE01825A8D
:101A40009440823391051CF486E10E94AB0C0F9008
:101A50000F90CF91DF9108950F931F93CF93DF9352
:101A60008AB590E00E94762C082F8093B00211E096
:101A70000DC088E10E94AB0C8AB590E00E94762CE4
:101A8000E12FF0E0E055FD4F80831F5F0E94FA07D1
:101A9000992787FD90950E94622C009731F48AB5B2
:101AA0008E3219F08AB58F3519F41C3028F3E1CF46
:101AB000E12FF0E0E055FD4F1082113099F4C02F76
:101AC000DD27C7FDD095CE010E946F2C009761F0F5
:101AD00083E08EBBC156D040CE01AA2797FDA095CA
:101AE000BA2F28C0143078F5013611F0043659F5B4
:101AF0008091B102992787FD9095C0978A30910512
:101B000010F52091B202822F992787FD9095C097FA
:101B10008A30910510F02223B1F4013611F083E1EF
:101B200001C082E18EBB80EB92E00E944C0890E005
:101B3000A0E0B0E08093A7029093A802A093A9022E
:101B4000B093AA0233C080EB92E06DEF73E041E006
:101B50000E941E0C882349F0E091A702F091A80290
:101B6000EB5CFB4FE491EEBB21C080EB92E065E6BD
:101B700072E041E00E941E0C882311F08EE013C039
:101B800080EB92E00E949806AA2797FDA095BA2FB5
:101B90008093A7029093A802A093A902B093AA02EF
:101BA000B7FD03C085E18EBB01C01EBADF91CF91A6
:101BB0001F910F910895EF92FF920F931F937B0156
:101BC0008C018091C102873018F089E00E94AB0C33
:101BD0008091C102E82FF0E0EE0FFF1FEE0FFF1F14
:101BE000EE53FD4FE082F182028313838F5F809377
:101BF000C1021F910F91FF90EF90089564E00E9441
:101C00008D0C08958091C102882319F489E00E9407
:101C1000FE0DE091C102E150E093C102F0E0EE0F51
:101C2000FF1FEE0FFF1FEE53FD4F60817181828118
:101C300093810895EF92FF920F931F93CF93DF93B9
:101C40008C0180E090E09C01200F311F44E02030A7
:101C50003407BCF40E944906EC018FEFCF3FD80750
:101C600081F0CE010E9435062FEF8F3F920711F4CD
:101C700080E094E09C012C1B3D0B201731071CF3E6
:101C800005C081E10E94FE0DC0E0D0E0CE01DF91F1
:101C9000CF911F910F91FF90EF900895682F82E0F0
:101CA0000E948D0C0895682F81E00E948D0C08958C
:101CB000803218F08EE00E94530E0895CF92DF928A
:101CC000EF92FF921F93CF93DF93182F6A017B014E
:101CD0000E94580E112349F481E594E0B701A60152
:101CE0000E94401A20E030E020C0C12FD0E0CC0F8D
:101CF000DD1FC55BDC4F60E472E48FE090E0A7017C
:101D000096010E94D42B2250304039832883812FA2
:101D100061E00E948304812F61E00E94A204888117
:101D200099810E94C20328813981C901DF91CF9135
:101D30001F91FF90EF90DF90CF9008951F93182F81
:101D40000E94580E10934A03112389F0E12FF0E00E
:101D5000EE0FFF1FE55BFC4F80819181009739F406
:101D6000812F40E855E260E070E00E945E0E1F9116
:101D70000895DF92EF92FF920F931F93CF93DF931B
:101D8000EC01ADE0EA2EF9E0FF2E08E71AE00E9430
:101D9000FA07882321F48CE00E94530E41C08AB5D3
:101DA000823251F40E94FA07DF91CF911F910F9177
:101DB000FF90EF90DF9008958AB58C3589F50E94E9
:101DC000FA07823771F083371CF48E3649F505C067
:101DD000843729F0883721F506C01ABD21C0FABC26
:101DE0001FC0EABC1DC00E94FA070E94AF078823EB
:101DF00099F08AB50E94ED0BD82E0E94FA070E9436
:101E0000AF07882349F08AB50E94ED0BD294E0EF2A
:101E1000DE22D80EDABC04C085E10E94530E0ABD52
:101E20008AB5FE010995B3CF85E10E94530E6AB5CC
:101E300070E080E090E00E94D8090E94F9090895BE
:101E4000EF92FF920F931F93CF93DF93EC010E94C9
:101E5000020E7B018C010E94020EDC01CB01C53217
:101E6000D10509F473C0C632D1052CF5C730D105B0
:101E700009F4ADC0C830D1056CF4C530D10509F402
:101E80008CC0C630D1050CF09CC0C430D10509F01F
:101E9000E8C079C0C930D10509F489C0C930D1057D
:101EA0000CF4A4C0CA30D10509F4C5C0CB30D105AB
:101EB00009F0D7C0CAC0CF32D10509F440C0C03341
:101EC000D1059CF4CA32D10599F1CB32D1052CF45D
:101ED000C632D10509F0C5C0A0C0CB32D105D1F0C2
:101EE000CD32D10509F0BDC01CC0CE33D10509F4F7
:101EF0003FC0CF33D1052CF4CC33D10509F0B1C0AC
:101F00002CC0CE35D10509F48FC0CC37D10509F0EE
:101F1000A8C07CC0BC01CD016E0D7F1D801F911F2C
:101F20009DC0BC01CD016E197F09800B910B96C03D
:101F3000BC01CD01A80197010E94A22B8FC0BC015A
:101F4000CD01A80197010E94F62B5DC0BC01CD0117
:101F5000A80197010E94F62B81C020E030E040E00C
:101F600050E08E159F05A007B1070CF04CC047C08C
:101F700020E030E040E050E0E816F9060A071B07D1
:101F80000CF041C03CC020E030E040E050E0E816FA
:101F9000F9060A071B07BCF132C020E030E040E040
:101FA00050E08E159F05A007B1076CF128C020E016
:101FB00030E040E050E08E159F05A007B107F9F42E
:101FC00022C00097A105B10531F460E00BC0009775
:101FD000A105B10531F460E0E114F104010511053A
:101FE00009F061E070E080E090E038C020E030E08F
:101FF00040E050E08E159F05A007B10721F421E0D5
:1020000030E040E050E0CA01B90128C0BC01CD0178
:102010006E297F29802B912B21C0BC01CD016E211F
:102020007F21802391231AC0BC01CD016E257F251D
:102030008027912713C0BC01CD0104C0660F771F14
:10204000881F991FEA94D2F709C0BC01CD0104C0D2
:102050009595879577956795EA94D2F70E94DB0D61
:1020600003C08AE00E94530EDF91CF911F910F9120
:10207000FF90EF900895682F80E00E948D0C0895E6
:1020800060E00E948D0C08959C01B901882777FDBE
:102090008095982F0E94DC098BE10E9440100895E2
:1020A0000E945F0980E00E94401008950E94FA0794
:1020B000992787FD9095A92FB92F8093A702909318
:1020C000A802A093A902B093AA0281E08EBB0E944D
:1020D000FA07873219F087E20E9450100E94FA072F
:1020E0000895CF93DF9380E090E00E943506EC01E5
:1020F0008FEFCF3FD807A9F0CE010E945F0A82E19F
:102100000E94780CCE010E945D06EC010E945F0ADD
:1021100082E20E945F090E94F909CE010E945D06D9
:10212000E4CFDF91CF910895EF92FF920F931F9329
:10213000CF93DF938C010E940B07C091A502D09131
:10214000A6022197D093A602C093A5020E94DE07A3
:102150001092AC021092AD021092AE021092AF0239
:1021600084E197E00E94B90E2091AC023091AD025B
:102170004091AE025091AF02211531054105510544
:10218000B1F1F80101900020E9F73197E01BF10B64
:10219000C90102968E0F9F1F0E941A0E7C0197FDA7
:1021A00026C0B8010E94CA06D093A602C093A50219
:1021B0000E94DE07F80101900020E9F73197E01B4B
:1021C000F10B0894E11CF11CEE0EFF1E00E010E084
:1021D000E092AC02F092AD020093AE021093AF0217
:1021E00088E297E00E94B90E80E00E942807DF9104
:1021F000CF911F910F91FF90EF900895DF93CF93B0
:10220000CDB7DEB72D970FB6F894DEBF0FBECDBFAA
:10221000CE01019660EB72E04DE050E00E946E2B23
:102220000E94BD078EB3823219F083E00E943B10FA
:10223000CE0101960E94941080E10E94880C0E94B9
:10224000BD072D960FB6F894DEBF0FBECDBFCF9160
:10225000DF9108950E94971381E391E00E94090B9A
:102260008AE10E94780C85E692E00E94090B0E94A8
:10227000F9090E94F9090E9471100895EF92FF92E6
:102280000F931F93DF93CF9300D00F92CDB7DEB79C
:102290000E94030D8EB38131F1F4E090A502F0901D
:1022A000A602F092A602E092A5020E94DE070E941A
:1022B000BD070E94C0166115710581059105B9F031
:1022C0008EB38A3319F08AE30E9450100E94BD0732
:1022D0000E94E312E6CF8EB38031B9F40E94BD07AD
:1022E0000E94C016611571058105910519F48FE0F2
:1022F0008EBB5FC18EB38A3319F08AE30E945010FF
:102300000E94BD070E94E31254C18EB38F3109F0C1
:102310004BC00E94BD070E94C016182F8EB38A338F
:1023200049F08AE369837A839B830E9450109B81E2
:102330007A816981E62EF72E012F192F17FF03C02E
:10234000EE24FF2487010E94BD078EB3853119F06A
:1023500086E00E943B100E94BD078EB38B3399F03C
:102360008EB38F3009F010C10EC08CE20E94501065
:10237000E114F1040105110531F00894E108F108B8
:1023800001091109E0CF8091A7029091A8020E9453
:10239000A8148EB38B3309F40CC18EB38F3009F4BB
:1023A00008C10E94BD07F5CF8EB3853121F08EB3F1
:1023B000882309F0EEC00E94BD078EB3843119F462
:1023C0000E94FE10F6C08EB38B3321F08EB38F3097
:1023D00009F0E4C08091A7029091A8020E94A8147D
:1023E000E8C00E94BD078EB3853119F088E10E94D4
:1023F000530E0E94BD078EB38C32E1F46091A702A8
:102400007091A8028091A9029091AA020E94DB0D0E
:102410000E94BD070E94C0160E94020EDC01CB0183
:1024200090684091AC025091AD026091AE02709103
:10243000AF0209C08091A7029091A802906840E085
:1024400050E060E070E00E94AF0CB3C08EB3893101
:1024500009F50E94BD078EB38A3219F40E9406095D
:102460008DC08EB38B3321F08EB38F3009F09AC0BC
:1024700080918B03882321F0E0918D03F0E095C0DB
:102480000E94060996C0EE0FFF1FE257FC4F118213
:1024900010828FC08EB38A3109F44DC08EB386315D
:1024A000A1F40E94BD078EB3853129F480EB92E040
:1024B0000E940B0763C08EB38A3219F40E940E0982
:1024C0005DC088E10E943B1059C08EB3883119F479
:1024D0000E94B80A6EC08EB38B3129F40E94BD07EA
:1024E0000E940D0A66C08EB38D3129F40E94BD078B
:1024F0000E9471105EC08EB38C3129F40E94BD071A
:102500000E942A1156C08EB38E3129F40E94BD0755
:102510000E94DA184EC08EB38A3399F582E00E9489
:10252000FA0B182F84E00E94FA0B7C0182E00E94D3
:10253000FA0B813019F40E9482073BC0882309F00E
:1025400038C0E114F10411F40E940E091E0D11C0EF
:1025500082E00E94FA0BF999FECF1FBAF2BCE1BCEF
:1025600080BD0FB6F894FA9AF99A0FBE0894E11C50
:10257000F11C1E1569F782E00E94FA0B0E94BD074C
:1025800018C00E949C1615C08EB38C3209F0EDCE97
:10259000EFCE8EB3873109F059CF23CF8BE30E9462
:1025A000501007C00E94C016FB01E430F10508F48A
:1025B0006ACF0F900F900F90CF91DF911F910F91E5
:1025C000FF90EF90089505C00E94BD078EB38F3035
:1025D00011F00E943E118EB38B33B1F30895DF9357
:1025E000CF9300D0CDB7DEB79A8389831092A4022F
:1025F0001092A30286EB93E00E940C2B8130910590
:1026000029F40E94060910924A0311C01092C102D7
:1026100089819A819093A6028093A5020E94DE0789
:102620000E94BD078EB38F3011F00E94E3120F900D
:102630000F90CF91DF910895CF93DF9380918C031A
:10264000882309F071C0C0E0D0E080918D038F5FD6
:1026500080938D03843010F010928D03E0918D03F0
:10266000F0E0EE0FFF1FE257FC4F80819181009751
:1026700009F455C00E945B039B01AC01E0918D03FE
:10268000F0E0DF01AA0FBB1FAA0FBB1FAA55BC4F6A
:102690008D919D910D90BC91A02D281739074A0767
:1026A0005B07E8F181E080938B03EE0FFF1FE25799
:1026B000FC4F80819181009719F481E00E94530EB4
:1026C000E0918D03F0E0EE0FFF1FE257FC4F808199
:1026D00091819F770E945D0690680E94EF120E9490
:1026E0005B039B01AC0180918D0390E0880F991FE3
:1026F000880F991FFC01EA55FC4F8A569C4FEC014C
:1027000088819981AA81BB81280F391F4A1F5B1FCD
:10271000208331834283538310928B0305C021961B
:10272000C430D10509F091CFDF91CF910895CF93B7
:10273000DF93CFE4D2E0CE0164EF71E04FE450E0EC
:102740000E945F2BCE010E94EF12DF91CF9108957E
:102750000F931F93DF93CF93CDB7DEB72D970FB6AF
:10276000F894DEBF0FBECDBF89E10E945F0CBC01B3
:102770008E010F5F1F4FC8014CE050E00E945F2B9D
:10278000C8010E94980697FD06C00E945D069068E9
:102790000E94EF1203C083E10E94780C2D960FB6C1
:1027A000F894DEBF0FBECDBFCF91DF911F910F9187
:1027B00008958FE492E090934E0280934D020E9420
:1027C000A81304C081E594E00E94BA1A81E594E060
:1027D0000E94A41A8823B1F70895AB01BC0181E5DA
:1027E00094E00E94401A0E94971387E10E945F0CB8
:1027F000BC018FE492E04FE450E00E945F2B8FE435
:1028000092E00E94980697FD04C08FE492E00E9437
:10281000EF120E94D913089560E076E980E090E01D
:102820000E94ED1308951F93CF93DF9381E594E009
:102830000E94A41A882309F47BC080914D029091D4
:102840004E0222E08E39920718F084E10E94AB0C10
:1028500081E594E00E94BA1A182F8D3021F08A3059
:1028600011F0803661F40E94F909E0914D02F09177
:102870004E0210828FE492E00E94EF1207C0833074
:1028800041F486E00E94880C0E9406090E94D91338
:102890004FC0823049F480E090918C03992309F471
:1028A00081E080938C0344C0883011F08F3701F5AC
:1028B00080914D0290914E0222E08F34920721F4D4
:1028C00087E00E945F0934C088E00E945F0980E2CF
:1028D0000E945F0988E00E945F09E0914D02F0913B
:1028E0004E023197F0934E02E0934D02108220C0C9
:1028F000853199F488E00E94880C0E94A813CFE4E7
:10290000D2E0CE010E94000A09900020E9F7219749
:10291000D0934E02C0934D020BC00E945F09E0911C
:102920004D02F0914E021193F0934E02E0934D024E
:102930000E941C13DF91CF911F9108950E941314E0
:1029400008950E94CF030E940C140E949E14FDCF94
:102950001F93CF93DF931EB397FD19C0C091A502BB
:10296000D091A6020E945D060E9445080E94BD0704
:102970000E94E3128EB38F3019F08CE00E943B105E
:10298000D093A602C093A5020E94DE071EBBDF9172
:10299000CF911F910895FF920F931F93CF93DF93D1
:1029A0001091A702F090A8020EB30E94BD07033158
:1029B00009F4AAC00431A8F40C3009F4C2C00D30E7
:1029C00030F4013021F1033009F036C129C00E3056
:1029D00009F47DC00E3008F4CCC0023109F02CC1DE
:1029E00081C0083209F4E1C0093238F4053109F434
:1029F00072C0013209F020C109C10D3209F4F1C0E1
:102A00000E3709F4FAC00B3209F016C1C9CF609134
:102A1000A7027091A8028091A9029091AA0209C10F
:102A20008EB38D3389F40E94BD070E94C016E12F3A
:102A3000F0E0EE0FFF1FEE0FFF1FEE51FD4F608322
:102A400071838283938336C08EB38C30B1F4C12FEF
:102A5000D0E0CC0FDD1FCC0FDD1FCE51DD4F6881E4
:102A600079818A819B810E94DB0D88819981AA816D
:102A7000BB810196A11DB11D18C08EB38D30D1F45C
:102A8000C12FD0E0CC0FDD1FCC0FDD1FCE51DD4FAD
:102A9000688179818A819B810E94DB0D888199817F
:102AA000AA81BB810197A109B10988839983AA836F
:102AB000BB8394C0E12FF0E0EE0FFF1FEE0FFF1F6E
:102AC000EE51FD4F6081718182819381B2C0812F6F
:102AD0000E94D216B4C00E94BD07812F9F2D0E9474
:102AE000A8141CC08EB38D3359F40E94BD070E94F8
:102AF000C0169B01AC01812FB9010E942A040EC0AF
:102B0000812F0E940C0416C08EB38D3381F40E9475
:102B1000BD070E94C016812F0E94A2046091AC02E2
:102B20007091AD028091AE029091AF0282C0812F70
:102B30000E94EE049C01B901882777FD8095982FAB
:102B400078C08EB3833019F08DE00E943B10E09185
:102B5000A702F0E0EE0FFF1FEE0FFF1FEE51FD4F3B
:102B600060817181828193816F5F7F4F8F4F9F4F13
:102B700017C08EB3833019F08DE00E943B10E091B6
:102B8000A702F0E0EE0FFF1FEE0FFF1FEE51FD4F0B
:102B9000608171818281938161507040804090405A
:102BA000608371838283938317C00E949C168091F7
:102BB000AB02813019F08EE00E943B108EB3893257
:102BC00019F08FE00E944E0E6091AC027091AD0240
:102BD0008091AE029091AF020E94DB0D0E94BD0772
:102BE0002EC00E94CB140E94020E90958095709585
:102BF00061957F4F8F4F9F4F1CC00E94CB140E9446
:102C0000020E609570958095909513C00E94CB142C
:102C10000E94020E9B01AC0160E070E080E090E059
:102C2000211531054105510521F461E070E080E096
:102C300090E00E94DB0D03C08EE00E94530EDF91F6
:102C4000CF911F910F91FF9008951F930E94CB1475
:102C50008EB38A3231F08EB38F3219F08EB3853253
:102C600061F41EB30E94BD070E94CB14812F9927E7
:102C700087FD90950E94200FEBCF1F9108951F9321
:102C80000E9425168EB38B3219F08EB38D3261F40B
:102C90001EB30E94BD070E942516812F992787FD2C
:102CA00090950E94200FEECF1F9108951F930E94D0
:102CB0003F168EB38B3019F08EB38A3061F41EB399
:102CC0000E94BD070E943F16812F992787FD90958E
:102CD0000E94200FEECF1F9108951F930E94561659
:102CE0000BC01EB30E94BD070E945616812F992764
:102CF00087FD90950E94200F0E949807882389F7EE
:102D00001F9108951F930E946D168EB3863231F085
:102D10008EB38C3719F08EB38E3561F41EB30E94DA
:102D2000BD070E946D16812F992787FD90950E94FF
:102D3000200FEBCF1F9108951F930E9482168EB330
:102D4000863019F08EB3873061F41EB30E94BD0740
:102D50000E948216812F992787FD90950E94200F4F
:102D6000EECF81E08093AB020E94020E6093AC0232
:102D70007093AD028093AE029093AF021F910895BD
:102D80000E949C168091AB02813019F08EE00E9467
:102D90003B106091AC027091AD028091AE029091B7
:102DA000AF0208958F929F92AF92BF92CF92DF921F
:102DB000EF92FF920F931F93DF93CF93CDB7DEB7C0
:102DC00068970FB6F894DEBF0FBECDBF082FE82F6F
:102DD000FF27E7FDF095EC5BFD4FE49019821A8226
:102DE0001B821C828EB38832D9F50E94BD0710E089
:102DF0008E2C992487FC90945E010894A11CB11C30
:102E000002C00E94BD078EB38932B1F0C12EDD240D
:102E1000C814D9048CF40E94C016F601EE0FFF1FEF
:102E2000EE0FFF1FEA0DFB1D648375838683978376
:102E30001F5F8EB38C3229F38EB3893219F08FE085
:102E40000E943B10812F90E0FF24E7FCF0948E1548
:102E50009F0519F08EE00E943B100E94BD0705C03F
:102E6000EE2019F088E20E945010E02FFF27E7FDC6
:102E7000F095E032F10508F081C1E25CFF4FEE0F02
:102E8000FF1F0590F491E02D0994ED80FE800F81E5
:102E900018852DC08D819E810E94C20372C10E943F
:102EA0005B0340C18D8169850E9483046AC18D8165
:102EB0000E94EE0454C18D8169850E94A20461C103
:102EC0006D817E818F8198850E94F1085AC168EEDC
:102ED00073E080E090E00E9498030E94030D88E177
:102EE0009CEFAFEFBFEFE80EF91E0A1F1B1F98EE15
:102EF000E91693E0F90690E0090790E019073CF71E
:102F0000C801B7010E9498033CC18D819E81AF81A9
:102F1000B885F999FECF92BD81BDF89A80B526C1DA
:102F20002D813E814F8158858985F999FECF1FBA41
:102F300032BD21BD80BD0FB6F894FA9AF99A0FBE42
:102F400020C181E594E00E94A41A10C181E594E0BB
:102F50000E94BA1A04C18091BD029091BE02A09154
:102F6000BF02B091C00205C12D813E814F815885BD
:102F700089859A85AB85BC85C5C02D813E814F81F1
:102F8000588589859A85AB85BC8582179307A407E8
:102F9000B5070CF0EEC0BBC06D817E818F81988536
:102FA00029853A854B855C85ED84FE840F851889DB
:102FB0000E94260BE6C0CE01825A9440D0C08D817B
:102FC0009E81AF81B88589839A83AB83BC83B7FF29
:102FD000D8C0B095A095909581959F4FAF4FBF4FAA
:102FE000C8C08D819E81AF81B885181619061A0652
:102FF0001B062CF481E090E0A0E0B0E0BAC000979E
:10300000A105B10509F4BDC08FEF9FEFAFEFBFEF92
:10301000B0C02091150130911601409117015091D7
:103020001801E0901901F0901A0100911B01109114
:103030001C01CA01B901F9E19695879577956795C5
:10304000FA95D1F76E0D7F1D801F911FE7E0220FCB
:10305000331F441F551FEA95D1F762277327842732
:103060009527609315017093160180931701909333
:1030700018017F77807090702D813E814F81588537
:103080000E94F62B69837A838B839C83D801C701C6
:1030900039E1B695A795979587953A95D1F78151DE
:1030A0009144A245B14227E0EE0CFF1C001F111F06
:1030B0002A95D1F78E259F25A027B1278093190146
:1030C00090931A01A0931B01B0931C015AC08D81EB
:1030D0000E940C0444C069857A858D810E942A046F
:1030E00050C02D813E814F81588589859A85AB8559
:1030F000BC85281739074A075B07DCF18D859E855B
:10310000AF85B889281739074A075B0794F5DA01B4
:10311000C9012FC02D853E854F8558898D816985D0
:103120000E943B0569837A838B839C832AC00D812F
:10313000802F61E00E9483041985812F61E00E9445
:103140008304802F612F4D8529890E94C20519C0F3
:1031500049855A856B857C858D810E945E0EAA27E4
:1031600097FDA095BA2F05C08091C10290E0A0E024
:10317000B0E089839A83AB83BC8303C088E10E945B
:10318000530E69817A818B819C810E94DB0D689648
:103190000FB6F894DEBF0FBECDBFCF91DF911F9168
:1031A0000F91FF90EF90DF90CF90BF90AF909F90E6
:1031B0008F9008951F938EB3833281F40E94BD07D0
:1031C0000E94C016162F8EB38A3319F08AE30E942C
:1031D00050100E94BD07812F0E949E0E8EB3823236
:1031E00051F48AB580931301109214018FE599E090
:1031F0000E94B90E73C00E949C168EB38A3309F0E8
:1032000070C00E94BD078EB3833009F089C08091E1
:10321000A7029091A802A091A902B091AA028731B9
:103220009105A105B10509F07BC06091AC027091D8
:10323000AD028091AE029091AF020E94D8094EC0BB
:103240008091A7029091A802A091A902B091AA0230
:1032500081309105A105B10509F066C06091AC020D
:103260007091AD028091AE029091AF020E94D4099C
:1032700035C08091A7029091A802A091A902B091B7
:10328000AA0288319105A105B10509F051C08091CC
:10329000AC020E945F0922C08EB30E945F09809138
:1032A000AC029091AD02A091AE02B091AF029C0130
:1032B000AD0121503040404050402093AC0230934B
:1032C000AD024093AE025093AF02181619061A06CB
:1032D0001B0614F303C08BE00E943B100E94BD0745
:1032E0000AC06091AC027091AD028091AE029091E3
:1032F000AF020E94DC098EB38B3319F08EB38F308E
:10330000E1F40E94F90908C00E94BD078EB38B3317
:1033100019F08EB38F30B1F410924A031F910895C3
:103320008EB3833009F48CCF8EB3833009F4A1CFF0
:103330008EB3813208F0B3CFCECF8EB38C3209F08A
:103340003ACFE2CF80E20E945F0935CF1F920F9201
:103350000FB60F9211242F933F934F935F936F9368
:103360007F938F939F93AF93BF93EF93FF9340917E
:10337000C60020914D0430914E04C901019660E8C9
:1033800070E00E94C12BBC0180914F0490915004C9
:103390006817790741F023533C4FF901408370933C
:1033A0004E0460934D04FF91EF91BF91AF919F91B7
:1033B0008F917F916F915F914F913F912F910F90DE
:1033C0000FBE0F901F9018958F92AF92CF92DF9201
:1033D000EF92FF920F931F93DF93CF93CDB7DEB79A
:1033E000FC0181E291E09183808373836283558342
:1033F00044833783268311870087F386E286D58648
:10340000C486A68687868D85808B8E85818BCF919D
:10341000DF911F910F91FF90EF90DF90CF90AF90D1
:103420008F9008958F92AF92CF92DF92EF92FF929A
:103430000F931F93DF93CF93CDB7DEB7FC0181E2EB
:1034400091E09183808373836283558344833783C0
:10345000268311870087F386E286D586C486A686F2
:1034600087868D85808B8E85818BCF91DF911F9193
:103470000F91FF90EF90DF90CF90AF908F900895D5
:10348000CF92DF92EF92FF920F931F93CF93DF9330
:10349000EC017A018B01CC80DD80CB01BA0122E006
:1034A00030E040E050E00E94F62BCA01B9016053C1
:1034B0007D4E8C4E9F4FA80197010E94F62BC901AB
:1034C000DA019C01AD012150304040405040232F93
:1034D000342F452F552747FD5A95F6012083E8855F
:1034E000F9851082EE81FF8181508083EA85FB851A
:1034F000808121E030E0A9010E8402C0440F551FF5
:103500000A94E2F7842B8083EA85FB858081A901F8
:103510000F8402C0440F551F0A94E2F7842B808366
:10352000EA85FB858081088802C0220F331F0A9438
:10353000E2F7822B8083DF91CF911F910F91FF9053
:10354000EF90DF90CF900895FC0122813381F90143
:10355000E058FF4F8081918180589F4F2E573F4FF9
:10356000F90120813181821B930B60E870E00E9499
:10357000C12B0895DC0112962D913C911397F9010E
:10358000EE57FF4F80819181D901A058BF4F4D91D7
:103590005C9111974817590719F42FEF3FEF0CC0B2
:1035A000280F391FD9012C91019660E870E00E9424
:1035B000C12B9183808330E0C9010895DC0112960C
:1035C0008D919C911397FC01E058FF4F8E579F4FB0
:1035D000DC018D919C911197918380830895FC016A
:1035E000A085B18521898C9190E0022E02C095952D
:1035F00087950A94E2F780FFF6CF0484F585E02DE5
:103600006083089581E291E0909352048093510485
:103610008DEC93E0909354048093530485EC90E0F8
:10362000909356048093550484EC90E09093580452
:103630008093570480EC90E090935A04809359044F
:1036400081EC90E090935C0480935B0486EC90E0C6
:1036500090935E0480935D0484E080935F0483E034
:103660008093600487E08093610485E08093620426
:103670000895DC01ED91FC910190F081E02D099518
:1036800008950E94391B08950F931F93CF93DF93E2
:10369000EC018B0105C00F5F1F4FCE010E94391B4B
:1036A000F80160816623B9F7DF91CF911F910F91E7
:1036B0000895CF93DF93EC016DE00E94391BCE019A
:1036C0006AE00E94391BDF91CF910895CF93DF9379
:1036D000EC010E94391BCE010E94591BDF91CF9152
:1036E0000895CF93DF93EC010E94441BCE010E940A
:1036F000591BDF91CF910895CF93DF93EC010E9486
:10370000391BCE010E94591BDF91CF9108952F9252
:103710003F924F925F926F927F928F929F92AF9261
:10372000BF92CF92DF92EF92FF920F931F93DF939E
:10373000CF93CDB7DEB7A2970FB6F894DEBF0FBE1A
:10374000CDBF2C015A016B01411551056105710571
:1037500021F460E30E94391B4CC0EE24FF24870152
:10376000622E7724882499241E010894211C311C80
:10377000C1018E0D9F1D9AA389A3C601B501A401A5
:1037800093010E94D42BE9A1FAA160830894E11C63
:10379000F11C011D111DC601B501A40193010E9478
:1037A000D42BA22EB32EC42ED52EA114B104C10445
:1037B000D104F1F6D801C7010197A109B109280E7A
:1037C000391E12C00894E108F10801091109F1013C
:1037D00060816A3010F4605D01C0695CC2010E94C2
:1037E000391B089421083108E114F1040105110581
:1037F00049F7A2960FB6F894DEBF0FBECDBFCF91AA
:10380000DF911F910F91FF90EF90DF90CF90BF90CD
:10381000AF909F908F907F906F905F904F903F9070
:103820002F9008952AE00E94871B0895CF93DF937D
:10383000EC010E94121CCE010E94591BDF91CF9116
:103840000895AB0160E070E00E94121C0895CF93D0
:10385000DF93EC01AB0160E070E00E94121CCE012E
:103860000E94591BDF91CF910895EF92FF920F9321
:103870001F93CF93DF93EC017A018B0177FF0BC08D
:103880006DE20E94391B10950095F094E094E11CC4
:10389000F11C011D111DCE01B801A7012AE00E94F3
:1038A000871BDF91CF911F910F91FF90EF900895AB
:1038B000CF93DF93EC010E94351CCE010E94591B6F
:1038C000DF91CF9108959B01A901662757FD60956F
:1038D000762F0E94351C0895CF93DF93EC01CB0126
:1038E000AC01662757FD6095762FCE010E94351CEE
:1038F000CE010E94591BDF91CF910895211531050A
:1039000021F4642F0E94391B08952A30310519F4DF
:103910000E94351C08950E94871B0895CF93DF9362
:10392000EC010E947E1CCE010E94591BDF91CF91B9
:1039300008958F929F92AF92BF92CF92DF92EF92B3
:10394000FF920F931F93CF93DF93EC016A017B01EA
:10395000122FCB01BA0120E030E040E050E00E949D
:103960005326882344F4CE016DE20E94391BF7FAF6
:10397000F094F7F8F09400E050E040E030E02FE3FE
:1039800011C0DA01F9016B2F742F8F2F922F20E0D5
:1039900030E040E251E40E947425562F472F382F23
:1039A000292F0F5F011768F3C701B601DA01F9018A
:1039B0002B2F342F4F2F5E2F0E944D247B01082F79
:1039C000A92E7F2D0E94A322B62ED72E882EC92E77
:1039D000CE014B2D5D2D682D7C2D0E94121C1123D4
:1039E00029F0CE0163E271E00E94441B6B2D7D2D16
:1039F000882D9C2D0E9435279B01AC016E2D7F2DBB
:103A0000802F9A2D0E941C2423C020E030E040E249
:103A100051E40E947A24F62EC72E082FE92E0E9428
:103A2000E1264B01AA2497FCA094BA2CCE01B50143
:103A3000A4010E94351CC501B4010E9483269B018C
:103A4000AC016F2D7C2D802F9E2D0E941C241150C7
:103A50001123D9F6DF91CF911F910F91FF90EF9035
:103A6000DF90CF90BF90AF909F908F90089522E00D
:103A70000E94991C0895CF93DF93EC010E94371D9B
:103A8000CE010E94591BDF91CF910895F999FECF85
:103A900072BD61BDF89A80B50895F999FECF1FBA3D
:103AA00072BD61BD40BD0FB6F894FA9AF99A0FBE87
:103AB00008950895FC01603DA9F0613D28F4603946
:103AC00059F0603CA1F40BC0603E19F0643F79F4FA
:103AD0000CC052A741A7089554A743A7089556A71D
:103AE00045A7089550AB47A7089552AB41AB089541
:103AF0006F3F19F4FC0154AB43AB0895613719F4DF
:103B0000FC0156AB45AB0895FC0150AF47AB08959F
:103B1000603F69F06F3F19F0613769F404C0FC0140
:103B200014AA13AA0895FC0116AA15AA0895FC0167
:103B300010AE17AA089540E050E00E945A1D089563
:103B4000FC01138214821582DC0180E016961C921F
:103B500016978F5F11968032C9F716A210A617A28A
:103B600003A8F4A9E02D309709F009950895FC0108
:103B700010820E94A01D0895FC0110820E94A01DC9
:103B8000089584E694E00E94B71D08958F929F9255
:103B9000AF92BF92CF92DF92EF92FF921F93CF939B
:103BA000DF93EB016A0149018DE061E00E9483042B
:103BB00010E0AA2497FCA094BA2CEE24D7FCE09441
:103BC000FE2C11C0C501B4010E9498038DE061E094
:103BD0000E94A204C701B6010E9498038DE060E034
:103BE0000E94A2041F5F812F90E08C179D0754F361
:103BF000DF91CF911F91FF90EF90DF90CF90BF901A
:103C0000AF909F908F900895CF93DF93EC018DE05C
:103C100061E00E948304CE0162E070E048EC50E075
:103C200020E931E00E94C61D6CE271E080E090E086
:103C30000E949803CE0162E070E041E050E024E091
:103C400030E00E94C61D6CE271E080E090E00E94CE
:103C50009803CE0160E070E048EC50E020E931E0EC
:103C60000E94C61DDF91CF9108950F931F93CF93AC
:103C7000DF938A01C1E5D4E0462F50E04F705070C9
:103C80004069662757FD6095762FCE0120E030E031
:103C90000E947E1CC80160E870E00E94C12BAC014C
:103CA000662757FD6095762FCE0120E030E00E9418
:103CB0007E1C000F012F001F110BA801662757FD66
:103CC0006095762FCE0120E030E00E947E1CDF91CF
:103CD000CF911F910F910895CF93DF93C1E5D4E069
:103CE000CE0149EF50E060E070E020E030E00E945B
:103CF0007E1CCE0142E050E060E070E020E030E069
:103D00000E947E1CCE0140E050E060E070E020E0C8
:103D100030E00E947E1CDF91CF91089581E594E010
:103D200047EF50E060E070E020E030E00E947E1C51
:103D3000089581E594E040EF50E060E070E020E01D
:103D400030E00E947E1C08950F931F93CF93DF9362
:103D50008C01C1E5D4E0AC01662757FD6095762F54
:103D60004F77507060707070CE0120E030E00E949C
:103D70007E1C000F012F001F110BA801662757FDA5
:103D80006095762F4F77507060707070CE0120E094
:103D900030E00E947E1CDF91CF911F910F9108951A
:103DA000CF92DF92FF920F931F93DF93CF930F92E7
:103DB000CDB7DEB7F42E122F032F69830E94991E10
:103DC0006981462F50E060E070E081E594E020E0FA
:103DD00030E00E947E1CC801492F582F6A0106C09E
:103DE000F60181916F0190E00E94A41E8C2D811B31
:103DF0008F15B0F30E948E1E0F90CF91DF911F910F
:103E00000F91FF90DF90CF9008959A01DA010D9005
:103E10000020E9F7AD0141505040421B530B0E9476
:103E2000D01E0895AB0161E70E94051F0895CF934E
:103E3000DF93EA01462F50E04F705070406E6627C6
:103E400057FD6095762F81E594E020E030E00E94F8
:103E50007E1CCE010E94A41EDF91CF91089581E5C2
:103E600094E00E94A41A90E00895AF92BF92CF927E
:103E7000DF92EF92FF920F931F93CF93DF93EC01AA
:103E80008B01F42EE22ECB0165E271E00E94882BBB
:103E90006C01C8016FE270E00E947D2B5C01C114CF
:103EA000D10459F00894A11CB11CA114B10429F04B
:103EB0008C2D8E5F8A1988830BC0D8010D9000204D
:103EC000E9F78A2F801BE82FEF5FE883A02EB12E41
:103ED000888190E00E94A6299C019A838983888129
:103EE000280F311DF9011082E981FA81F082E98100
:103EF000FA81E18289819A81488150E042505040A4
:103F00000296B5010E946E2BDF91CF911F910F9108
:103F1000FF90EF90DF90CF90BF90AF9008951F93E8
:103F2000CF93DF93EC018881882351F10E94991E81
:103F300081E594E049E750E060E070E020E030E0A7
:103F40000E947E1CE981FA8181E594E060810E94F3
:103F5000391BE981FA8181E594E061810E94391B76
:103F600012E009C0E981FA81E10FF11D808190E042
:103F70000E94A41E1F5F88811817A0F30E948E1E46
:103F8000DF91CF911F9108950F931F93CF93DF93EC
:103F9000EC018E81813731F08937B1F5CE010E9475
:103FA0008F1F3CC08DA99EA90097C1F18FA198A534
:103FB000019762E070E00E94C12B062F10E0C8015B
:103FC0000E94A629E82FF92F0E0F1F1F31E015C000
:103FD000DE01A30FB11D16964C914083A32FAF5F56
:103FE000BE016A0F711DDB0116962C91169727955D
:103FF00022272795240F21933E5FE017F10741F711
:10400000EDA9FEA909950AC0EFA9F8AD309731F0E6
:104010006FA16150AE01495F5F4F0995DF91CF916C
:104020001F910F910895CF93DF93EC0181E594E008
:104030000E94BA1A2EA1222399F0873F910529F4F4
:104040001EA2CE010E94C41F93C02FA138A5FE015D
:10405000E20FF31F86832F5F3F4F38A72FA388C03F
:104060002B81222309F446C0803891050CF042C010
:1040700021502B83FE01E20FF11D8683222309F0DC
:1040800077C08C81882309F473C0803D49F1813D5C
:1040900028F4803959F0803C59F51FC0803E19F052
:1040A000843F31F513C0E9A5FAA502C0EBA5FCA534
:1040B0003097F1F06E8170E07695762F66277795D0
:1040C00067958F81680F711D8D8111C0E9A9FAA9CB
:1040D000309771F06E818F8109C0EDA5FEA502C0F9
:1040E000EFA5F8A9309721F06E818D8170E00995D8
:1040F0001C823EC0803F910514F09C0105C09C01CC
:10410000207F30708F708D83203E3105F1F0213E8D
:10411000310554F4203C3105D1F0203D3105B9F092
:104120002039310529F511C0243F310571F0253FB3
:10413000310524F4203F3105D9F40DC0293F310564
:1041400099F02F3F3105A1F40BC082E001C081E05E
:104150008B832C830DC081E08EA318A61FA208C0FC
:10416000CE010E94A01D04C084E694E00E946C1E53
:10417000DF91CF910895EF92FF920F931F93CF930A
:10418000DF93EC017A018B010E94041E81E594E02B
:10419000B801A7010E94401A6CE271E080E090E053
:1041A0000E949803CE010E946C1ECE010E948F1FB8
:1041B000DF91CF911F910F91FF90EF900895CF93D2
:1041C000DF93EC0181E594E040E052EC61E070E0C7
:1041D0000E94401ACE010E94041E6CE271E080E051
:1041E00090E00E949803CE010E946C1EDF91CF9157
:1041F00008952FB7F89482E0809380008AE180933D
:10420000810088EB9BE090938900809388009093D5
:104210008B0080938A0080E593EC909387008093D5
:104220008600EFE6F0E08081887F80832FBF0895CD
:104230000895FC0110828FEF81830895FC011082A4
:104240008FEF81830895DF92EF92FF920F931F9378
:10425000CF93DF93EC018B0177FF03C000E010E008
:1042600005C0653B710514F004EB10E00983DA80AA
:104270006B8170E06D197109882777FD8095982F03
:1042800020E431E040E050E00E94A22B202F30E0FB
:1042900040E050E00E94A22B24EB30E040E050E0F0
:1042A0000E94F62B79018A016D2D70E080E090E08C
:1042B00020E431E040E050E00E94A22BE60EF71E21
:1042C000081F191FC801B70128E030E040E050E0A6
:1042D0000E94F62B8881893029F43093890020933D
:1042E000880006C08A3021F430938B0020938A0026
:1042F000DF91CF911F910F91FF90EF90DF90089584
:10430000FC0181810895FC018081893031F4809124
:104310009D04882351F081E008958A3011F080E0F7
:10432000089580919E04811181E00895CF93DF93D9
:10433000EC018881893059F410929D0480918000AD
:104340008F738093800089E060E00E9483048881FD
:104350008A3059F410929E04809180008F7C809363
:1043600080008AE060E00E948304DF91CF9108958D
:10437000CF93DF93EC01FB01CA01AB0149505040E0
:104380004230510510F080E037C060E170E00E94DB
:10439000C12B6A83C90160E170E00E94C12B6B836D
:1043A000E8838FEF89838E2F60E00E94A2048881CA
:1043B00061E00E94830480919D04882331F4809100
:1043C0009E04882311F40E94F9208881893041F4E9
:1043D00081E080939D04809180008F73806809C084
:1043E0008A3049F481E080939E04809180008F7C24
:1043F00080628093800081E0DF91CF91089540E258
:1044000052E020E639E00E94B82108952F923F92B1
:104410004F925F926F927F928F929F92AF92BF92D4
:10442000CF92DF92EF92FF920F931F93DF93CF9380
:10443000CDB7DEB73B014C0119012A016D897E8998
:104440008F89988D6A197B098C099D09621A730AF4
:10445000840A950AA40193010E94A22BE218F30892
:1044600004091509A80197010E94F62B2A0D3B1D8E
:104470004C1D5D1DB901CA01CF91DF911F910F91B4
:10448000FF90EF90DF90CF90BF90AF909F908F9074
:104490007F906F905F904F903F902F900895089578
:1044A00070E0382F20E0622B732BCB010895EF9240
:1044B000FF920F931F937B018C016115710581059C
:1044C000910529F420E030E040E050E00FC00E9468
:1044D000FE2AA80197010E94F62B572F482F392F4B
:1044E000862F952FA42FB32F9C01AD01B901CA01CE
:1044F0001F910F91FF90EF900895EF92FF920F930D
:104500001F937B018C01621773078407950764F47E
:10451000CA01B9016E197F09800B910B0E945722C5
:10452000E60EF71E081F191FB701C8011F910F9152
:10453000FF90EF900895009729F0BC0180E090E093
:104540000E94032B0895EF92FF920F931F937B011C
:104550008C0120E030E040E05FE40E9423268823C5
:104560008CF0C801B70120E030E040E05FE40E9439
:104570001C240E94E1269B01AC01205030404040A9
:10458000504806C0C801B7010E94E1269B01AC015A
:10459000B901CA011F910F91FF90EF900895A0E01B
:1045A000B0E0E5EDF2E20C94272CFC012B01EA01CE
:1045B0008081823008F43AC1DB019C91923008F48A
:1045C00034C1843069F4943009F030C1918111967E
:1045D0008C911197981709F429C1EAE2F1E026C1FC
:1045E000943009F422C19230A9F4823009F01EC13E
:1045F0009F0188E0D9010D909D01DA010D92AD0176
:104600008150C1F7D20111968C9111979181892324
:10461000898309C1823009F408C182819381DB0159
:1046200012964D915C911397E480F5800681178175
:104630001496AD90BD90CD90DC9017979C01241BF3
:10464000350BB90137FF04C066277727621B730B50
:10465000603271050CF062C0121613066CF535015C
:104660004601062E04C096948794779467940A9422
:10467000D2F721E030E040E050E004C0220F331FC9
:10468000441F551F6A95D2F721503040404050409A
:104690002A213B214C215D21211531054105510580
:1046A00021F021E030E040E050E059016A01A62805
:1046B000B728C828D9283DC021153105D1F1860F6A
:1046C000971F37014801062E04C09694879477946B
:1046D00067940A94D2F721E030E040E050E004C053
:1046E000220F331F441F551F6A95D2F721503040C7
:1046F000404050402E213F214023512321153105B8
:104700004105510521F021E030E040E050E0790121
:104710008A01E628F728082919290BC048175907E4
:104720002CF0CA01EE24FF24870103C0AA24BB2475
:1047300065012181F2013181231709F447C0222349
:1047400049F0A60195012E193F09400B510B790143
:104750008A0104C0EA18FB080C091D0917FD0CC0EA
:1047600019829B838A83EC82FD820E831F838C8156
:104770009D81AE81BF8117C021E029839B838A83FD
:1047800010950095F094E094E11CF11C011D111DA1
:10479000EACF880F991FAA1FBB1F2A813B81215096
:1047A00030403B832A839C01AD0121503040404082
:1047B00050402F3F6FEF36076FEF46076FE3560706
:1047C00040F38C839D83AE83BF830BC029839B837F
:1047D0008A83EA0CFB1C0C1D1D1DEC82FD820E83DE
:1047E0001F8383E088832C813D814E815F8157FF49
:1047F0001AC0C901AA2797FDA095BA2F81709070A1
:10480000A070B0705695479537952795822B932BBE
:10481000A42BB52B8C839D83AE83BF838A819B8120
:1048200001969B838A83FE0101C0F201CF01CDB7BF
:10483000DEB7E0E10C94432CA0E2B0E0E2E2F4E267
:104840000C94312C69837A838B839C832D833E83E4
:104850004F835887E9E0EE2EF12CEC0EFD1ECE01C1
:104860000196B7010E94D8288E010F5E1F4FCE011E
:104870000596B8010E94D8288A8991E089278A8BF9
:10488000C701B801AE01475E5F4F0E94CF220E9470
:104890000728A096E6E00C944D2CA0E2B0E0E3E5FA
:1048A000F4E20C94312C69837A838B839C832D836F
:1048B0003E834F835887F9E0EF2EF12CEC0EFD1E5E
:1048C000CE010196B7010E94D8288E010F5E1F4FBE
:1048D000CE010596B8010E94D828C701B801AE01E3
:1048E000475E5F4F0E94CF220E940728A096E6E015
:1048F0000C944D2CA0E2B0E0E0E8F4E20C94252CFE
:1049000069837A838B839C832D833E834F8358876F
:10491000CE010196BE01675F7F4F0E94D828CE016D
:104920000596BE016F5E7F4F0E94D8289985923010
:1049300088F089898230C8F0943019F4823051F4BB
:1049400004C0843029F4923081F48AE291E0C6C038
:10495000923049F480E02A859A89291381E08A8778
:10496000CE010996BBC0823049F480E02A859A893D
:10497000291381E08A8BCE014196B0C06D847E847C
:104980008F849888AD88BE88CF88D88C60E070E02E
:1049900080E090E0A0E0B0E0EE24FF24870120E07A
:1049A00030E040E050E0F301E170F0703097C9F082
:1049B0002A0D3B1D4C1D5D1D8E0D9F1DA01FB11F9F
:1049C0002224332421012A153B054C055D0528F4DA
:1049D000E1E02E2E312C412C512C820D931DA41D73
:1049E000B51DEE0CFF1C001F111FD7FE09C0E1E032
:1049F0002E2E312C412C512CE228F3280429152984
:104A00006F5F7F4F6032710549F0AA0CBB1CCC1C54
:104A1000DD1C9694879477946794C5CF6B897C89C5
:104A2000EB85FC856E0F7F1F6E5F7F4F7C8F6B8FDA
:104A30001A8E7A856A89761711F061E06A8F6B8D1C
:104A40007C8D10C0FC01E170F070309729F0569514
:104A50004795379527955068B695A795979587956B
:104A60006F5F7F4FB7FDEECF0CC0880F991FAA1F55
:104A7000BB1F57FD8160220F331F441F551F61501C
:104A800070408030E0E09E07E0E0AE07E0E4BE0763
:104A900060F36B8F7C8F6FE7E62EF12C012D112DCB
:104AA000E822F9220A231B2360E4E616F10401053B
:104AB000110561F487FD0AC0211531054105510535
:104AC00029F0805C9F4FAF4FBF4F80788D8F9E8FB6
:104AD000AF8FB8A383E0898FCE0149960E94072843
:104AE000A096E2E10C94412CA8E1B0E0EAE7F5E2FF
:104AF0000C942D2C69837A838B839C832D833E8336
:104B00004F8358878E01075F1F4FCE010196B80172
:104B10000E94D82881E1E82EF12CEC0EFD1ECE017A
:104B20000596B7010E94D8289985923008F484C070
:104B30008989823010F487017FC02A853A8923272A
:104B40002A87943011F0923031F4981709F071C02F
:104B50000AE211E071C0843039F41D861E861F867A
:104B6000188A1C861B8668C0823019F484E0898705
:104B700063C08B859C852B893C89821B930B9C870A
:104B80008B872D853E854F855889AD88BE88CF8817
:104B9000D88C2A153B054C055D0538F4220F331FD0
:104BA000441F551F01979C878B8760E070E0E12CC4
:104BB000F12C012DA0E41A2F80E090E0A0E0B0E0FD
:104BC0002A153B054C055D0540F08E299F29A02B39
:104BD000B12B2A193B094C095D0916950795F794E5
:104BE000E794220F331F441F551F6F5F7F4F6F31B4
:104BF000710531F76FE7E62EF12C012D112DE8221A
:104C0000F9220A231B2360E4E616F10401051105CD
:104C100061F487FD0AC0211531054105510529F0D0
:104C2000805C9F4FAF4FBF4F80788D879E87AF8747
:104C3000B88B8E01075F1F4FC8010E940728689636
:104C4000EAE00C94492CA8E1B0E0E9E2F6E20C9429
:104C5000312C69837A838B839C832D833E834F839E
:104C6000588789E0E82EF12CEC0EFD1ECE0101964E
:104C7000B7010E94D8288E010F5E1F4FCE01059606
:104C8000B8010E94D8288985823040F08989823015
:104C900028F0C701B8010E94472901C08FEF68962C
:104CA000E6E00C944D2CA8E1B0E0E9E5F6E20C94C6
:104CB000312C69837A838B839C832D833E834F833E
:104CC000588789E0E82EF12CEC0EFD1ECE010196EE
:104CD000B7010E94D8288E010F5E1F4FCE010596A6
:104CE000B8010E94D8288985823040F089898230B5
:104CF00028F0C701B8010E94472901C081E06896E9
:104D0000E6E00C944D2CA8E0B0E0E9E8F6E20C9463
:104D10002F2C7B018C0183E08983D801C701882770
:104D2000B7FD83959927AA27BB278A83E114F1044D
:104D30000105110519F482E089833BC08823B1F095
:104D400080E0E81680E0F80680E0080780E81807B1
:104D500029F460E070E080E09FEC2FC01095009592
:104D6000F094E094E11CF11C011D111D8EE1C82E90
:104D7000D12CDC82CB82ED82FE820F831887C801A2
:104D8000B7010E94AE279C01215030401216130635
:104D900084F4022E04C0EE0CFF1C001F111F0A94A5
:104DA000D2F7ED82FE820F831887C21AD30ADC8203
:104DB000CB82CE0101960E9407282896E8E00C9449
:104DC0004B2CACE0B0E0E7EEF6E20C94352C6983B6
:104DD0007A838B839C83CE010196BE016B5F7F4FEC
:104DE0000E94D8288D81823061F1823050F1843068
:104DF00021F48E81882351F12EC02F81388537FD13
:104E000020C06E812F3131051CF06623F9F023C0DC
:104E10008EE190E0821B930B29853A854B855C855A
:104E200004C056954795379527958A95D2F76623FE
:104E3000B1F050954095309521953F4F4F4F5F4FC2
:104E40000EC020E030E040E050E009C02FEF3FEF1F
:104E50004FEF5FE704C020E030E040E050E8B901E8
:104E6000CA012C96E2E00C94512CA8E0B0E0EBE3F0
:104E7000F7E20C942F2C7B018C011A8261157105CD
:104E80008105910519F482E0898360C083E08983FC
:104E90008EE1C82ED12CDC82CB82ED82FE820F8384
:104EA0001887C801B7010E94AE279C0121503040ED
:104EB00037FF39C0EE27FF27E21BF30B40E050E03D
:104EC00060E070E081E090E0A0E0B0E00E2E04C071
:104ED000880F991FAA1FBB1F0A94D2F70197A10937
:104EE000B1098E219F21A023B1230097A105B1050F
:104EF00021F041E050E060E070E004C016950795B5
:104F0000F794E794EA95D2F7E42AF52A062B172BB3
:104F1000ED82FE820F8318878EE190E0821B930B57
:104F20009C838B8313C02115310581F0022E04C0B0
:104F3000EE0CFF1C001F111F0A94D2F7ED82FE82B7
:104F40000F831887C21AD30ADC82CB82CE01019666
:104F50000E9407282896E8E00C944B2CAF92BF9251
:104F6000CF92DF92EF92FF920F931F937B018C0100
:104F700080E0E81680E0F80681E0080780E0180786
:104F800088F48FEFE816F1040105110531F028F0DF
:104F900088E090E0A0E0B0E017C080E090E0A0E002
:104FA000B0E012C080E0E81680E0F80680E0080774
:104FB00081E0180728F088E190E0A0E0B0E004C0AC
:104FC00080E190E0A0E0B0E020E230E040E050E09E
:104FD000281B390B4A0B5B0B5701680104C0D694A0
:104FE000C794B794A7948A95D2F7F501EE5CFE4F6B
:104FF0008081281B310941095109C9011F910F9175
:10500000FF90EF90DF90CF90BF90AF900895CF9238
:10501000DF92EF92FF920F931F93FC012481358161
:105020004681578101818081823020F440618FEF79
:1050300090E0A4C0843009F49BC0823019F480E071
:1050400090E098C0211531054105510519F480E023
:1050500090E094C0828193816FEF823896070CF0C4
:1050600059C062E87FEF681B790B6A3171052CF03B
:1050700020E030E040E050E02AC069017A01062ECD
:1050800004C0F694E794D794C7940A94D2F781E0C9
:1050900090E0A0E0B0E004C0880F991FAA1FBB1FDA
:1050A0006A95D2F70197A109B10982239323A4231A
:1050B000B5230097A105B10521F081E090E0A0E0C3
:1050C000B0E09C01AD012C293D294E295F29DA0170
:1050D000C9018F779070A070B07080349105A105E0
:1050E000B10539F427FF09C0205C3F4F4F4F5F4F98
:1050F00004C0215C3F4F4F4F5F4F80E090E0203075
:1051000060E0360760E0460760E4560748F181E05A
:1051100090E026C0803891055CF581589F4F7FE76D
:10512000C72ED12CE12CF12CC222D322E422F5226D
:1051300060E4C616D104E104F10439F427FF09C084
:10514000205C3F4F4F4F5F4F04C0215C3F4F4F4F9C
:105150005F4F57FF05C056954795379527950196A0
:1051600097E056954795379527959A95D1F706C0BC
:105170008FEF90E020E030E040E050E0782F77952E
:1051800077277795142F1F77602F67956627679588
:105190008695F12FF72BE82FE62B622F732F8F2F99
:1051A0009E2F1F910F91FF90EF90DF90CF90089569
:1051B000FC01DB01208131818281482F4F7750E053
:1051C000982F991F9927991F6381862F880F892B04
:1051D00090E0661F6627661F11966C9311970097E3
:1051E00069F5211531054105510511F482E02FC003
:1051F00082E89FEF13969C938E93129767E0220F9D
:10520000331F441F551F6A95D1F783E08C930DC05F
:10521000220F331F441F551F12968D919C91139797
:10522000019713969C938E931297203080E0380755
:1052300080E0480780E4580758F322C08F3F91056B
:1052400079F4211531054105510519F484E08C9359
:10525000089544FF03C081E08C9312C01C9210C0DB
:105260008F57904013969C938E93129783E08C9364
:1052700087E0220F331F441F551F8A95D1F75064D2
:1052800014962D933D934D935C9317970895EF9249
:10529000FF920F931F93FC01DB018081823008F4A1
:1052A00047C09C91923008F443C0843051F481810E
:1052B0009430A1F511962C91119730E0281B3109FB
:1052C0003FC0943021F0823031F49230B9F1119620
:1052D0008C9111972BC08181923001F111969C9194
:1052E00011978917D9F44281538112962D913C91DF
:1052F00013972417350794F042175307BCF0E48046
:10530000F5800681178114962D913D914D915C9108
:1053100017972E153F054007510718F4882341F0D1
:105320000AC0E216F3060407150740F4882319F0B3
:1053300021E030E005C02FEF3FEF02C020E030E079
:10534000C9011F910F91FF90EF900895CF93DF93C4
:105350008230910510F482E090E0A091A104B09118
:10536000A204FD0120E030E0C0E0D0E020C0408198
:1053700051814817590761F482819381209719F070
:105380009B838A833AC09093A2048093A10435C082
:105390008417950738F42115310519F04217530782
:1053A00008F49A01EF0152814381E52FF42F3097E1
:1053B000F1F621153105B9F1A901481B590B44300B
:1053C000510508F4C901E0E0F0E02BC04D915C917B
:1053D00011974217530701F58217930781F412962C
:1053E0008D919C911397309719F09383828304C019
:1053F0009093A2048093A104FD0132964FC0281B14
:10540000390BFD01E20FF31F81939193225030403D
:1054100011963C932E9342C0FD0152814381A52FEA
:10542000B42F109799F620919F043091A004211574
:10543000310541F420913402309135023093A004BB
:1054400020939F04209136023091370221153105B7
:1054500041F42DB73EB74091320250913302241BE4
:10546000350BE0919F04F091A004E217F307A0F43C
:105470002E1B3F0B2817390778F0AC014E5F5F4FAA
:105480002417350748F04E0F5F1F5093A004409338
:105490009F048193919302C0E0E0F0E0CF01DF919F
:1054A000CF910895CF93DF93009709F451C0FC0189
:1054B000329713821282A091A104B091A204109796
:1054C00051F140E050E0AE17BF0748F412968D91BD
:1054D0009C911397AD01009719F1DC01F4CFB383D0
:1054E000A283EF0129913991CE01820F931FA81752
:1054F000B90771F48D919C911197820F931F0296B9
:105500009183808312968D919C91139793838283CC
:105510004115510529F4F093A204E093A10418C0A9
:10552000DA011396FC93EE9312972D913D91A20F01
:10553000B31FEA17FB0761F480819181820F931FEB
:105540000296EA0199838883828193819B838A836F
:10555000DF91CF910895A0E0B0E0E1EBFAE20C9486
:105560002D2CEC01E880F9800A811B81E114F10403
:105570000105110541F484E2E82E89EDF82E8BE552
:10558000082F87E0182FC801B7012DE133EF41E064
:1055900050E00E94F62B27EA31E440E050E00E9400
:1055A000A22B5B016C01C801B7012DE133EF41E093
:1055B00050E00E94F62BCA01B9012CEE34EF4FEFF8
:1055C0005FEF0E94A22B9B01AC012A0D3B1D4C1DDD
:1055D0005D1D57FF04C02150304040405048288393
:1055E00039834A835B835F77B901CA01CDB7DEB7E0
:1055F000EAE00C94492C0E94AB2A089588E392E0DB
:105600000E94AB2A08956093380270933902809308
:105610003A0290933B020895DC012D923D924D9207
:105620005D926D927D928D929D92AD92BD92CD9242
:10563000DD92ED92FD920D931D93CD93DD93FF913D
:10564000EF918DB78D938EB78D938FB78D93ED932B
:10565000FD93882799270994DC01CB0181309105BE
:10566000811D2D903D904D905D906D907D908D9021
:105670009D90AD90BD90CD90DD90ED90FD900D9101
:105680001D91CD91DD91ED91FD910D90F894FEBFAE
:105690000FBEEDBFED91FD910994FB01DC018D91F1
:1056A000059080190110D9F3990B0895FC0105901C
:1056B0000020E9F7809590958E0F9F1F0895FB01BC
:1056C000DC014150504048F005900D920020C9F790
:1056D00001C01D9241505040E0F70895FB01DC01EC
:1056E0004150504048F001900D920020C9F701C090
:1056F0001D9241505040E0F70895FC0181E090E098
:105700000190061609F4CF010020D1F70197089502
:10571000FB0151915523A9F0BF01DC014D914517C3
:105720004111E1F759F4CD010190002049F04D916C
:1057300040154111C9F3FB014111EFCF81E090E029
:1057400001970895629FD001739FF001829FE00D41
:10575000F11D649FE00DF11D929FF00D839FF00DF0
:10576000749FF00D659FF00D9927729FB00DE11D9C
:10577000F91F639FB00DE11DF91FBD01CF01112479
:10578000089597FB092E07260AD077FD04D049D04B
:1057900006D000201AF4709561957F4F0895F6F7B2
:1057A000909581959F4F0895A1E21A2EAA1BBB1BCD
:1057B000FD010DC0AA1FBB1FEE1FFF1FA217B307DD
:1057C000E407F50720F0A21BB30BE40BF50B661FF3
:1057D000771F881F991F1A9469F7609570958095B7
:1057E00090959B01AC01BD01CF01089597FB092E57
:1057F00005260ED057FD04D0D7DF0AD0001C38F4A0
:1058000050954095309521953F4F4F4F5F4F0895EC
:10581000F6F790958095709561957F4F8F4F9F4FCC
:105820000895AA1BBB1B51E107C0AA1FBB1FA617E7
:10583000B70710F0A61BB70B881F991F5A95A9F739
:1058400080959095BC01CD0108952F923F924F9283
:105850005F926F927F928F929F92AF92BF92CF9200
:10586000DF92EF92FF920F931F93CF93DF93CDB709
:10587000DEB7CA1BDB0B0FB6F894DEBF0FBECDBF81
:1058800009942A88398848885F846E847D848C8452
:105890009B84AA84B984C884DF80EE80FD800C815B
:1058A0001B81AA81B981CE0FD11D0FB6F894DEBF3E
:1058B0000FBECDBFED010895EE0FFF1F0590F491CF
:1058C000E02D0994911106C080538A5010F0865C37
:1058D00006C0089599278827089585FDFBCF80622B
:1058E0009111F8CF81568A51E0F7089591110895EA
:1058F00081548A5108F4805E855A0895F894FFCF48
:10590000018D087F0B2C0DCD08140F56100000C818
:10591000089808FFFFFECAEFBEEFBEADDE00000034
:1059200000EF1A2E002E63707000000000000000CF
:10593000000000010202030303030404040404043E
:105940000404050505050505050505050505050509
:1059500005050606060606060606060606060606E9
:1059600006060606060606060606060606060606D7
:1059700006060707070707070707070707070707B9
:1059800007070707070707070707070707070707A7
:105990000707070707070707070707070707070797
:1059A0000707070707070707070707070707070787
:1059B0000707080808080808080808080808080869
:1059C0000808080808080808080808080808080857
:1059D0000808080808080808080808080808080847
:1059E0000808080808080808080808080808080837
:1059F0000808080808080808080808080808080827
:105A00000808080808080808080808080808080816
:105A10000808080808080808080808080808080806
:105A200008080808080808080808080808080808F6
:0C5A300008082000A30400000100000092
:00000001FF
